:020000040000FA
:020000002E28A8
:08000800DE00030E8301AC00D1
:100010000A08AD008A011F281030AE000310A40D9D
:10002000A50D0310A00DA10D031C1C282308A50776
:100030002208A4070318A50AAE0B0E2808002E08F4
:10004000AF002008A6002108A7002208A800230866
:10005000A9002408AA002508AB003C2883168113B8
:10006000373095009F0183129F0107309900831656
:100070008510851505100F298B1C72288B10101008
:10008000BB153808B000B1013008A0003108A1004C
:100090001930A200A3010C202408B2002508B300E7
:1000A0003209B4003309B500A100FA303407A000CA
:1000B0000318A10A200883128E0021088F000C105B
:1000C000FA303802031D6828DD105D088500842899
:1000D0000C303802031D7028DD145D08850084286B
:1000E000101484280C1C8428BB1D7F28DD145D0897
:1000F0008500BB11F1308E00FF308F008328DD10AA
:100100005D08850010100C102608A0002708A1002B
:100110002808A2002908A3002A08A4002B08A5008B
:100120002F08AE002D088A002C0E8300DE0E5E0E16
:100130000900C10083169B001C141A080800BF00A8
:1001400083169B0040089A001C158B1355309D00A8
:10015000AA309D009C148B171C119C18AD28080018
:100160000C3039020319C928031CC92800000000FB
:10017000FB30A000C630A1000A128A11A10BBC28D6
:100180000A128A11A00BBA280000B9033908B80076
:10019000B028000000009B30A0001730A1008B3079
:1001A000A2000A128A11A20BD1280A128A11A10BED
:1001B000CF280A128A11A00BCD2800000000FA30C7
:1001C00039020319F8280318F82800000000FB3052
:1001D000A000C630A1000A128A11A10BEB280A1256
:1001E0008A11A00BE9280000B90A3908B800DF28F5
:1001F000000000009B30A0001730A1008B30A2004F
:100200000A128A11A20B00290A128A11A10BFE28D8
:100210000A128A11A00BFC2800000000B028DD1093
:100220005D0883128500B8015D105D08850000300F
:100230009920B600FA30360203192329031C23291A
:100240007D30B90025293608B90001309920B60063
:100250000230360203193029031C3029B701322934
:100260003608B7003708031D3829FA30B80044298A
:100270003703031D3E290C30B80044293908B80063
:100280005D145D0883128500BB103B103B11BB1150
:100290008316011383121010101390111015901073
:1002A000CF301005303890008E018F010C1083166E
:1002B0000C140B160B178B178312851DB02083129D
:1002C00085195F2900000000AD30A000C630A100F4
:1002D0000A128A11A10B68290A128A11A00B662939
:1002E000000000000000000000000000000000000E
:1002F000000085195F296430BA00851D8129BC1171
:100300008229BC153A083C1603193C12BC16BC19CC
:100310003C1EBC12BC1E9D29000000007430A000D1
:100320005530A1000A128A11A10B92290A128A11D2
:10033000A00B90290000BA037D293A08031DE52986
:1003400002303702031DE2293B1DA8293B11A929D0
:100350003B158519062A3B1DB6290C3039020319B5
:10036000BE29031CBE29B903BB14BE29FA303902C9
:100370000319BE290318BE29B90ABB143908B800ED
:100380000330BA00851DC6293D12C7293D163A081B
:10039000BD160319BD123D173D1ABD1E3D133D1F6D
:1003A000A929000000007430A0005530A1000A12F5
:1003B0008A11A10BD7290A128A11A00BD529000096
:1003C000BA03C2298519062AE2293708031DF02934
:1003D0000130B7005D105D0885000C30B800052ABB
:1003E0003703031DFB290230B7005D145D0885004B
:1003F0003908B800052A02303702031D052AB70163
:100400005D105D088500FA30B8003B14BB1C0D2A56
:100410003908C00000309F20BB103B1C5F29370803
:0A042000C00001309F203B105F294F
:02400E00823FEF
:00000001FF
